:020000001828BE
:080008008E00030E8D0083162B
:100010008B1C102883128618B3288B100B1683169E
:100020000B18A62083120D0E83008E0E0E0E0900F3
:1000300083128B1308308900831608148312000082
:100040000808081E3428003089000310153E84007B
:100050000830A300831608148312000008088000EB
:10006000840A890AA30B2A28831601138113061612
:100070008616061786140614861106110512051039
:100080008510051185118312850186110611003036
:1000900092000B108B100B168B158B1706087039FE
:1000A0008C0003108C0C8C0C8C0C30308C07A62030
:1000B000E0210130AF001530840000308000840A58
:1000C0008000840A8000153084000008013A03197A
:1000D0007C280008023A031985280008033A03190E
:1000E00084280008043A0319A42817308400000863
:1000F000003A031DA52863281630840000080B224F
:1001000084030030800063286328163084000008D0
:10011000013A03193C220008023A0319352200086B
:10012000083A0319422200080C3A03194522000834
:10013000103A031958220008143A03194A221530BC
:100140008400003080006328632863288312060837
:1001500070398C0003108C0C8C0C8C0C30308C079C
:100160000B108B15080083129F2112100F18121408
:100170000F100F0803110C06031DC728CB211218FE
:10018000D928012983128B100B1683161028D92128
:10019000061CC828861CC828FA3091000130861C2D
:1001A0000030061C0030910BCF289100111CC8288C
:1001B000C2289F21CB210F0893009319E82807300C
:1001C00013050310153E840000089000B321C228D7
:1001D0004C309000B32165309000B3216430900022
:1001E000B32131309000B32136309000B32131304B
:1001F0009000B3212E309000B32130309000B32115
:10020000C2289F21CB210F0893009F21CB210F08EB
:100210009400E03013059200003003111206031918
:100220002E292030120603193629403012060319F0
:10023000402960301206031955298030120603192F
:100240006F29A030120603197B29C030120603194A
:100250008C29E030120603199E29C22807301305A5
:100260000310153E840014088000C2281530840055
:100270000830910014088000840A910B3A29C228A2
:100280000730130589000310153E8400000888001C
:100290008316081555308900AA3089008814081182
:1002A000081E502908128312C2280030890003104A
:1002B000153E840008309100000888008316081558
:1002C00055308900AA30890088140811081E662953
:1002D00008128312890A840A910B5C29C22807300C
:1002E000130589000310153E840083160814831239
:1002F00008088000C228003089000310153E8400E1
:100300000830910083160814831208088000840ABC
:10031000890A910B8229C228083089001030130500
:1003200088008316081555308900AA308900881482
:100330000811081E992908128312C228C2288F01A9
:10034000083091008618A229861CA429061CA92918
:10035000AC2903108F0DB02903108F0D0F14B02995
:10036000910BA22908000830910083160610831211
:100370008618B829861CBA29900D031CC029C229E9
:100380000610C4290614C429910BB829D921831653
:100390000614831208008618CB29861CCD29061066
:1003A0008316061083128618D32983160614831227
:1003B00008008618D929861CDB298618DD29080043
:1003C0003C30A500A530A400A40BE429A50BE2292C
:1003D0002030FA210C30FA210630FA210130FA21BE
:1003E00008000830A500A530A400A40BF529A50B32
:1003F000F3290800AE00F1212E0E0F3905128611E7
:100400000615850006112E080F39051286110615EE
:10041000850006110800AD0009302F0603192522BA
:1004200031302F0603193522F1212D0E0F39051217
:1004300086150615850006112D080F39051286153B
:10044000061585000611AF0A08002030B0001430F0
:10045000FA21AF0AB00B272A08002030B000103074
:10046000FA21AF03B00B2F2A08000130AF00023091
:10047000FA210C30FA2108000130AF00FA210C30CB
:10048000FA2108000830FA2108000130AF000C30D2
:10049000FA2108001430FA21AF0A09302F06031997
:1004A000252231302F06031935220C30FA2108009D
:1004B0001030FA21AF0328302F0603192D22003007
:0C04C0002F06031935220C30FA21080029
:00000001FF
